:030000000202B643
:0100030032CA
:06000B00C2A9112B01A0A7
:0100130032BA
:01001B0032B2
:0400230010984032BF
:01002B0032A2
:05003300D211C2DC3215
:01003B003292
:02004300210793
:01004B003282
:060053005391BFD20332FD
:01005B003272
:10006300D21132C0E0C0D0C082C083C08675860082
:10007300E510B45A08E511B41B03020095851082FC
:10008300851183E599F0A385821085831175080096
:10009300D207D086D083D082D0D0D0E032D21732EC
:1000A300C0E0C0F0C083C082C092758A36758CF8F8
:1000B300BC00010C1C0508DA287A0A120295BD005F
:1000C300010D1DBE00010E1EDB177B0ABF00010FD1
:1000D3001F050912067BE530B405067530011206CB
:1000E30042D092D082D083D0F0D0E0D2A9227A0A33
:1000F3007B0A5389F0438901758A30758CF843A8CC
:1001030082D28C22C0E0C0D0C082C083C0F0C09233
:10011300C00175D000907FA8E003F5F003B406009A
:1001230040239406907FAA10E003907FA9033160D7
:100133005391EFF0316BD001D092D0F0D083D082C5
:10014300D0D0D0E032316B907FA8E00303316090D0
:100153007FABF5F074EF5291E5F0F080D904832280
:100163000102040810204080E5F090017173218999
:10017300416C416C21952198416C219C416C416CEF
:10018300416C41B441B5C22A12089D7402907FB4F8
:10019300F022D22A2222753200C3E5319532601053
:1001A300A932759213907F0051768932907FB5F012
:1001B300227902907FB6516DE510B45A06E511B469
:1001C300130122753005120642758600907E8085E4
:1001D300128485138575F000758601E0A38584126A
:1001E300858513758600F0A305F0C3E5109584702B
:1001F30007C3E51195856009E5F0B44000500E8012
:10020300D775105A75111375125A751313E5F090BB
:100213007FB7F022907FC6E030E10122907FC7E0F4
:100223006046907F9AE054107005D21402026B75F9
:100233003005120642907FC7E0F5F0907E40E02043
:10024300D005C29B02024CD29BF599A3C0F075F076
:10025300C8209903D5F0FA75F00AD5F0FDD0F0C2A5
:1002630099D5F0DA907FC7F02222E030E104D0E0A4
:10027300D0E022B4320040027432C0E0F5F0E3F083
:10028300A309D5F0F9D0E022F5F0E0F3A309D5F006
:10029300F9227902907FB8516D907E00E524F0A396
:1002A3007400F0A3F0A3F0907FB97404F0752400F8
:1002B300222222907F924402F075D000785F76006C
:1002C300D8FC75813F1203D411F1120ACC120784B2
:1002D30012085912074B120876907F9E7400F09013
:1002E3007F9BE023235403F521120520758E00D252
:1002F300147530021206427F051203C2BF00FA755D
:1003030030051206427F051203C2BF00FA753001A1
:100313001206427F051203C2BF00FA7530031206AC
:100323004275105A75111375125A75131330110350
:100333001205C11203CA20070512021731B41203B2
:10034300C21205BD302AE612088B80E1616D61801F
:10035300619661AC75F000907F9AE0A2E192F1A200
:100363000292F0E5F02390034F73C3E509950AC3A6
:1003730094024008120642D20285090A22C3E50903
:10038300950AC39430400B75F000120629C202850A
:10039300090A22C3E509950AC39430400B75F0306E
:1003A300120629D20285090A22C3E509950AC394D4
:1003B30002400B75F000120629C20285090A223099
:1003C300170411A3C21722C3E508940A4002C20707
:0E03D3002275A80075E80075F80075B800C224
:1003E100DD7480907FD6F0C2DCD2DD907F94E04452
:1003F10040F0D2ECC2DBD2AF22901008912063F022
:10040100FF55F0F022C0E0C2DCD0E022912065F07F
:10041100F0229120E5F0F022800271FA90400A85E5
:1004210083F043829075837FE022E045F0F022E57E
:10043100F064FFF5F0E055F0F02212046E907F9821
:10044100E0440A54FBF022907F9475F0BF9130751F
:10045100F040912B907F9D75F0BD912B75F05291DD
:100461003022907F9775F0A0912B914822907F9533
:1004710075F00E913075F030912B907F9E75F00ED6
:10048100912B75F030913022907F9875F00E912B61
:1004910075F0049130916E227F1E907F9A71C2E0B7
:1004A10030E1030204D771C2BF00030204D771C255
:1004B100907F9AE020E4E67DFA71C2E030E1030228
:1004C10004D771C2BD00030204D771C2907F9AE0C4
:1004D10030E4E67400227401229148916E907F9776
:1004E10075F0A09130907F9875F00A913075F00405
:1004F100912B22907F947440F0907F957400F0903E
:100501007F9D74BDF0907F9E74FFF0907F97740083
:10051100F0907F987400F07F0A71C2BF00FB2290B7
:100521007F9775F001912B2291F491899163913B11
:10053100B12022C203D2EAC2039148916E907F9703
:1005410075F0A09130907F9875F00A913075F004A4
:10055100912B91997027C203907F9875F004913087
:1005610075F008912B91997014907F9775F0A09177
:100571002B7530017D0A71C2BD00FB8000907F9711
:1005810075F0A0912B907F9875F004913075F0086B
:10059100912B907F9575F003912B22753003229159
:1005A100F491DAB120B1341206427F1E907F9AE0B5
:1005B10030E1012271C2BF00F3C214222014E022F3
:1005C100C2EC7530041206427D0A71C2BD00FB9077
:1005D1007F9AE030E10D91F4753003120642C210AA
:1005E100020622907F9AE020E605D2120205F2D29D
:1005F10013753001120642907F9AE054107002B1D7
:10060100A0301209C2127402F52402061730131128
:10061100C2137401F524753001120642020622D27A
:1006210010C211C2DBD2EC22C083C082C0E0907F35
:100631009CE0443063F03065F0F0D0E0D082D083AC
:1006410022E530B4011C75F010D12922E530B40146
:100651001175F0EFD12922E530B4010675F0EFD123
:100661002922B4020675F020D12922B4030675F0BF
:1006710000D1292275F030D12922907F9AE030E112
:100681000D301013C210753003D142D21122201047
:1006910006D214D210D211228322120103020102C6
:1006A10010002C085A400000000110018322094665
:1006B10080000101002702832209000000000300DD
:1006C10000048322070500400281058322070500FB
:1006D10010020105832207400010038205832204D2
:1006E100040903120A3D83221803586972636F6D6E
:1006F10020496E632E120A3D832244035553422D35
:100701004F4E4C5920524558203630303020446FDE
:10071100636B696E672053746174696F6E120A3D71
:1007210083221003524558444F434B120A3D832202
:100731000E033030303030303030303030308322C2
:100741000300008322030000E422740A1207F9F86F
:0E0751001207B97407B85A08900731741AF0ED
:10075F0074201207F97833759207790612083EF262
:10076F000812083CF20812080CD9F11207B97403E9
:10077F0090069DF02274001207F912080C9006A53E
:10078F00F0F812080C9006A4F0F9803312080C90C0
:10079F0006A3F012080C547F9006A2F0D20612089E
:1007AF000CB4102912080CB4022312080212080C00
:1007BF00907FA5E04440F07E0A71C2BE00FB22B8D4
:1007CF004507B91604D22C80C3C22C80BFF1B9746F
:1007DF000512081274101208207402120820200645
:1007EF00CF748812082080C874074480120812A39F
:1007FF00E0800A120824907FA5E04420F01208241C
:10080F00A3E0222344A0F5F0907FA5E04480F0E51B
:10081F00F0907FA6F0907FA57EFA1203C2E020E051
:10082F00E120E203BE00F3D0E0D0E08083E5F0C426
:10083F00F5F0540F2430B43A004002240722C3E2EB
:10084F009430B40A0040029407227401907FACF0F8
:10085F007400A3F07409A3F07407907FDEF07403A3
:10086F00A3F0C2DCD2DD22907FD6740AF07E9612FE
:10087F0003C2BE00FA7406F043E80122438701C2A7
:10088F002A22907FB4E020E304907FC5F022907F6E
:10089F00E8E0547FB40002801FB40202805E54600F
:1008AF00B44003020A5A22907FEAE0B4014D900748
:1008BF0043E054FD45F0F022907FE9E0B4060302D7
:1008CF00097BB4000690073F0209F8B40809E43029
:1008DF002F0274010209E2B4090F907FEAE070035E
:1008EF00C22F22B40115D22F22B4030675F00202D3
:1008FF0008B6B4010675F0000208B622907FE9E051
:10090F00B4000F1209465401900748F090074402B3
:10091F0009F8B403071209464401F022B401171273
:10092F00094654FEF0E5F0540730F7024410907F6B
:10093F00D7F04420F02222907FECE0F5F0547F6056
:10094F000CB4021230F71F2320F702241024B4F541
:10095F008275837FE02240EFB4030320CDE9B40614
:10096F000050032088E1D0E0D0E080CA907FEBE018
:10097F00900749B40103900699B402028008B403AA
:10098F000280260209FA9006ADD2281209FA9006C3
:10099F00B81209EB9006C31209EB9006CC1209EBC3
:1009AF009006D51209EB020A0B907FEAE0900749F7
:1009BF0070039006DEB401039006E4B4020D9007B5
:1009CF001E80069006F630CD02E5F0B403039007C3
:1009DF002C8018907F00F074010201AF120A2F854E
:1009EF003182758313D2288008D229120A2F9013CF
:1009FF0000120A0E8582311028226020020199749C
:100A0F0001120A2C6016F5F0302907C229120A2CA0
:100A1F0015F0F0A3E5F0120A2CD5F0F622020A2BFE
:100A2F008582F0E583900A2DF0A3E5F0F0220532E0
:100A3F00B40102F532E532B40400400E30E0069402
:100A4F000503240422D0E0D0E0E422E0C0E0C03B64
:100A5F00C03CC03D907FEAE0F53CA3E0F53DA3E04C
:100A6F00753B00120A7ED03DD03CD03BD0E022D265
:100A7F0001907FE9E0B48015900AB07436F0900AC7
:100A8F00AE7400F0A374E1F0900AAB21F8B4810BBF
:100A9F00900AB4020AA8900ABD21F82283220740C7
:100AAF003836000006832207820383820181832266
:100ABF000D820585820484820383820181C28E7533
:0E0ACF008DFF907F95E04403F07598D0E58987
:100ADD00540F4460F58975C80053877FD2ACD2BCE2
:050AED00D2ACD28E2204
:00000001FF
